BL51 BANKED LINKER/LOCATER V6.20                                                        06/05/2009  10:43:05  PAGE 1


BL51 BANKED LINKER/LOCATER V6.20, INVOKED BY:
D:\KEIL\C51\BIN\BL51.EXE ch375.obj, uart.obj, nRF2401.obj TO mou RAMSIZE (256)


MEMORY MODEL: SMALL


INPUT MODULES INCLUDED:
  ch375.obj (CH375)
  uart.obj (UART)
  nRF2401.obj (NRF2401)
  D:\KEIL\C51\LIB\C51S.LIB (?C_STARTUP)
  D:\KEIL\C51\LIB\C51S.LIB (?C?CLDPTR)
  D:\KEIL\C51\LIB\C51S.LIB (?C_INIT)


LINK MAP OF MODULE:  mou (CH375)


            TYPE    BASE      LENGTH    RELOCATION   SEGMENT NAME
            -----------------------------------------------------

            * * * * * * *   D A T A   M E M O R Y   * * * * * * *
            REG     0000H     0008H     ABSOLUTE     "REG BANK 0"
            DATA    0008H     0002H     UNIT         _DATA_GROUP_
            DATA    000AH     0001H     UNIT         ?DT?UART
                    000BH     0015H                  *** GAP ***
            BIT     0020H.0   0000H.1   UNIT         ?BI?NRF2401
                    0020H.1   0000H.7                *** GAP ***
            DATA    0021H     0019H     UNIT         ?DT?CH375
            IDATA   003AH     0001H     UNIT         ?STACK

            * * * * * * *   C O D E   M E M O R Y   * * * * * * *
            CODE    0000H     0003H     ABSOLUTE     
                    0003H     0020H                  *** GAP ***
            CODE    0023H     0003H     ABSOLUTE     
                    0026H     07DAH                  *** GAP ***
            CODE    0800H     008CH     UNIT         ?C_C51STARTUP
            CODE    088CH     0061H     UNIT         ?PR?MAIN?CH375
            CODE    08EDH     0053H     UNIT         ?PR?NRF2401_INIT?NRF2401
            CODE    0940H     0029H     UNIT         ?CO?CH375
            CODE    0969H     0024H     UNIT         ?PR?_SPI_SENDBYTE?NRF2401
            CODE    098DH     0020H     UNIT         ?PR?INITUART?UART
            CODE    09ADH     001EH     UNIT         ?C_INITSEG
            CODE    09CBH     001EH     UNIT         ?PR?_PRINTS?UART
            CODE    09E9H     001DH     UNIT         ?PR?SPI_RCVBYTE?NRF2401
            CODE    0A06H     001BH     UNIT         ?PR?_PRINTHEX?UART
            CODE    0A21H     0019H     UNIT         ?C?LIB_CODE
            CODE    0A3AH     0011H     UNIT         ?PR?SETRXMODE?NRF2401
            CODE    0A4BH     0010H     UNIT         ?CO?UART
            CODE    0A5BH     000DH     UNIT         ?CO?NRF2401
            CODE    0A68H     000CH     UNIT         ?PR?SERIALPORT?UART
            CODE    0A74H     000AH     UNIT         ?PR?_SENDTOCOMPORT?UART



OVERLAY MAP OF MODULE:   mou (CH375)

BL51 BANKED LINKER/LOCATER V6.20                                                      06/05/2009  10:43:05  PAGE 2



SEGMENT                             DATA_GROUP 
  +--> CALLED SEGMENT             START    LENGTH
-------------------------------------------------
?C_C51STARTUP                     -----    -----
  +--> ?PR?MAIN?CH375
  +--> ?C_INITSEG

?PR?MAIN?CH375                    0008H    0002H
  +--> ?PR?INITUART?UART
  +--> ?CO?CH375
  +--> ?PR?_PRINTS?UART
  +--> ?PR?NRF2401_INIT?NRF2401
  +--> ?PR?SETRXMODE?NRF2401
  +--> ?PR?_PRINTHEX?UART
  +--> ?PR?SPI_RCVBYTE?NRF2401

?PR?_PRINTS?UART                  -----    -----
  +--> ?PR?_SENDTOCOMPORT?UART

?PR?NRF2401_INIT?NRF2401          -----    -----
  +--> ?CO?NRF2401
  +--> ?PR?_SPI_SENDBYTE?NRF2401

?PR?_PRINTHEX?UART                -----    -----
  +--> ?CO?UART
  +--> ?PR?_SENDTOCOMPORT?UART



SYMBOL TABLE OF MODULE:  mou (CH375)

  VALUE           TYPE          NAME
  ----------------------------------

  -------         MODULE        CH375
  C:0000H         SYMBOL        _ICE_DUMMY_
  D:00A0H         PUBLIC        P2
  D:00B0H         PUBLIC        P3
  D:00D8H         PUBLIC        ADCSTAT
  D:00A8H         PUBLIC        IE
  D:00B8H         PUBLIC        IP
  D:00E8H         PUBLIC        I2CCON
  D:00E8H         PUBLIC        DCON
  C:088CH         PUBLIC        main
  D:0021H         PUBLIC        RcvFifo
  D:0098H         PUBLIC        SCON
  D:0088H         PUBLIC        TCON
  B:00B0H.3       PUBLIC        DR1
  D:00F8H         PUBLIC        SPICON
  D:00C8H         PUBLIC        T2CON
  D:00D0H         PUBLIC        PSW
  D:00C0H         PUBLIC        WDCON
  -------         PROC          MAIN
  -------         DO            
  D:0008H         SYMBOL        te
  D:0009H         SYMBOL        tmp
BL51 BANKED LINKER/LOCATER V6.20                                                      06/05/2009  10:43:05  PAGE 3


  -------         ENDDO         
  C:088CH         LINE#         17
  C:088CH         LINE#         18
  C:088CH         LINE#         23
  C:088FH         LINE#         24
  C:089AH         LINE#         35
  C:089DH         LINE#         38
  C:08A0H         LINE#         40
  C:08A0H         LINE#         41
  C:08A0H         LINE#         42
  C:08A2H         LINE#         43
  C:08A5H         LINE#         44
  C:08A5H         LINE#         45
  C:08B0H         LINE#         46
  C:08B5H         LINE#         47
  C:08B8H         LINE#         48
  C:08B8H         LINE#         49
  C:08C2H         LINE#         50
  C:08CBH         LINE#         53
  C:08CEH         LINE#         54
  C:08D3H         LINE#         58
  C:08D6H         LINE#         59
  C:08DBH         LINE#         62
  C:08DEH         LINE#         63
  C:08E3H         LINE#         66
  C:08E6H         LINE#         67
  C:08EBH         LINE#         73
  C:08EBH         LINE#         76
  -------         ENDPROC       MAIN
  -------         ENDMOD        CH375

  -------         MODULE        UART
  C:0000H         SYMBOL        _ICE_DUMMY_
  D:00A0H         PUBLIC        P2
  D:00B0H         PUBLIC        P3
  C:09CBH         PUBLIC        _Prints
  B:00A8H.7       PUBLIC        EA
  D:00D8H         PUBLIC        ADCSTAT
  C:0A68H         PUBLIC        SerialPort
  D:00A8H         PUBLIC        IE
  C:0A4BH         PUBLIC        HexTable
  B:00A8H.4       PUBLIC        ES
  D:00B8H         PUBLIC        IP
  B:0098H.0       PUBLIC        RI
  B:0098H.1       PUBLIC        TI
  D:00E8H         PUBLIC        I2CCON
  D:00E8H         PUBLIC        DCON
  D:0099H         PUBLIC        SBUF
  D:0087H         PUBLIC        PCON
  D:0098H         PUBLIC        SCON
  D:0089H         PUBLIC        TMOD
  D:0088H         PUBLIC        TCON
  C:0A06H         PUBLIC        _PrintHex
  C:0A74H         PUBLIC        _SendToComport
  D:00D7H         PUBLIC        PLLCON
  D:000AH         PUBLIC        Sending
  D:008DH         PUBLIC        TH1
BL51 BANKED LINKER/LOCATER V6.20                                                      06/05/2009  10:43:05  PAGE 4


  D:00F8H         PUBLIC        SPICON
  D:008BH         PUBLIC        TL1
  C:098DH         PUBLIC        InitUART
  B:0088H.6       PUBLIC        TR1
  B:0098H.4       PUBLIC        REN
  D:00C8H         PUBLIC        T2CON
  D:00D0H         PUBLIC        PSW
  D:00C0H         PUBLIC        WDCON
  -------         PROC          INITUART
  C:098DH         LINE#         25
  C:098DH         LINE#         26
  C:098DH         LINE#         27
  C:0990H         LINE#         28
  C:0992H         LINE#         29
  C:0995H         LINE#         30
  C:0998H         LINE#         31
  C:099BH         LINE#         33
  C:099EH         LINE#         34
  C:09A1H         LINE#         35
  C:09A4H         LINE#         36
  C:09A6H         LINE#         37
  C:09A8H         LINE#         38
  C:09AAH         LINE#         39
  C:09ACH         LINE#         40
  -------         ENDPROC       INITUART
  -------         PROC          SERIALPORT
  C:0A68H         LINE#         45
  C:0A68H         LINE#         47
  C:0A6BH         LINE#         48
  C:0A6BH         LINE#         49
  C:0A6DH         LINE#         50
  C:0A6EH         LINE#         52
  C:0A6EH         LINE#         53
  C:0A70H         LINE#         54
  C:0A73H         LINE#         55
  C:0A73H         LINE#         56
  -------         ENDPROC       SERIALPORT
  -------         PROC          _SENDTOCOMPORT
  D:0007H         SYMBOL        d
  C:0A74H         LINE#         60
  C:0A74H         LINE#         61
  C:0A74H         LINE#         62
  C:0A77H         LINE#         63
  C:0A79H         LINE#         64
  C:0A7DH         LINE#         65
  -------         ENDPROC       _SENDTOCOMPORT
  -------         PROC          _PRINTS
  D:0001H         SYMBOL        pd
  D:0005H         SYMBOL        line_feed
  C:09CBH         LINE#         70
  C:09CBH         LINE#         71
  C:09CBH         LINE#         72
  C:09D1H         LINE#         73
  C:09D1H         LINE#         74
  C:09D4H         LINE#         75
  C:09DBH         LINE#         76
  C:09DDH         LINE#         77
BL51 BANKED LINKER/LOCATER V6.20                                                      06/05/2009  10:43:05  PAGE 5


  C:09E0H         LINE#         78
  C:09E0H         LINE#         79
  C:09E5H         LINE#         80
  C:09E8H         LINE#         81
  C:09E8H         LINE#         82
  -------         ENDPROC       _PRINTS
  -------         PROC          _PRINTHEX
  D:0006H         SYMBOL        x
  C:0A06H         LINE#         139
  C:0A08H         LINE#         140
  C:0A08H         LINE#         143
  C:0A14H         LINE#         144
  C:0A1CH         LINE#         145
  -------         ENDPROC       _PRINTHEX
  -------         ENDMOD        UART

  -------         MODULE        NRF2401
  C:0000H         SYMBOL        _ICE_DUMMY_
  C:0A5CH         PUBLIC        nRF2401Addr1
  B:00A0H.0       PUBLIC        PWR_UP
  C:0A61H         PUBLIC        nRF2401Addr2
  D:00A0H         PUBLIC        P2
  D:00B0H         PUBLIC        P3
  D:00D8H         PUBLIC        ADCSTAT
  B:00A0H.1       PUBLIC        CE
  B:00A0H.3       PUBLIC        CLK1
  D:00A8H         PUBLIC        IE
  C:09E9H         PUBLIC        SPI_RcvByte
  B:00A0H.2       PUBLIC        CS
  D:00B8H         PUBLIC        IP
  D:00E8H         PUBLIC        I2CCON
  D:00E8H         PUBLIC        DCON
  D:0098H         PUBLIC        SCON
  D:0088H         PUBLIC        TCON
  C:08EDH         PUBLIC        nRF2401_Init
  D:00F8H         PUBLIC        SPICON
  B:0020H.0       PUBLIC        RX2_EN
  C:0A66H         PUBLIC        CH1DataLen
  C:0A67H         PUBLIC        CH2DataLen
  C:0A3AH         PUBLIC        SetRXMode
  D:00C8H         PUBLIC        T2CON
  C:0A5BH         PUBLIC        nRF2401AddrLen
  C:0971H         PUBLIC        _SPI_SendByte
  D:00D0H         PUBLIC        PSW
  B:00A0H.4       PUBLIC        Data
  D:00C0H         PUBLIC        WDCON
  -------         PROC          L?0023
  -------         ENDPROC       L?0023
  -------         PROC          _SPI_SENDBYTE
  D:0007H         SYMBOL        ch
  -------         DO            
  D:0006H         SYMBOL        i
  -------         ENDDO         
  C:0971H         LINE#         102
  C:0971H         LINE#         103
  C:0971H         LINE#         106
  C:0973H         LINE#         107
BL51 BANKED LINKER/LOCATER V6.20                                                      06/05/2009  10:43:05  PAGE 6


  C:0973H         LINE#         108
  C:0977H         LINE#         109
  C:097BH         LINE#         111
  C:097DH         LINE#         113
  C:0981H         LINE#         114
  C:0982H         LINE#         115
  C:0984H         LINE#         116
  C:0985H         LINE#         117
  C:0986H         LINE#         118
  C:0988H         LINE#         119
  C:098CH         LINE#         120
  -------         ENDPROC       _SPI_SENDBYTE
  -------         PROC          NRF2401_INIT
  -------         DO            
  D:0005H         SYMBOL        i
  -------         ENDDO         
  C:08EDH         LINE#         123
  C:08EDH         LINE#         124
  C:08EDH         LINE#         127
  C:08EFH         LINE#         129
  C:08F1H         LINE#         130
  C:08F3H         LINE#         132
  C:08F9H         LINE#         134
  C:08FFH         LINE#         136
  C:0901H         LINE#         137
  C:0901H         LINE#         138
  C:090AH         LINE#         139
  C:090CH         LINE#         141
  C:090EH         LINE#         142
  C:090EH         LINE#         143
  C:0917H         LINE#         144
  C:0919H         LINE#         146
  C:0928H         LINE#         149
  C:092BH         LINE#         150
  C:092FH         LINE#         152
  C:0934H         LINE#         154
  C:0939H         LINE#         156
  C:093BH         LINE#         157
  C:093DH         LINE#         159
  C:093FH         LINE#         160
  -------         ENDPROC       NRF2401_INIT
  -------         PROC          SPI_RCVBYTE
  -------         DO            
  D:0006H         SYMBOL        i
  D:0007H         SYMBOL        ch
  -------         ENDDO         
  C:09E9H         LINE#         167
  C:09E9H         LINE#         168
  C:09E9H         LINE#         169
  C:09EBH         LINE#         170
  C:09EDH         LINE#         171
  C:09EFH         LINE#         172
  C:09F1H         LINE#         173
  C:09F1H         LINE#         175
  C:09F5H         LINE#         176
  C:09F7H         LINE#         177
  C:09F8H         LINE#         178
BL51 BANKED LINKER/LOCATER V6.20                                                      06/05/2009  10:43:05  PAGE 7


  C:09F9H         LINE#         179
  C:09FBH         LINE#         180
  C:09FEH         LINE#         181
  C:0A01H         LINE#         183
  C:0A03H         LINE#         184
  C:0A05H         LINE#         186
  C:0A05H         LINE#         187
  -------         ENDPROC       SPI_RCVBYTE
  -------         PROC          SETRXMODE
  C:0A3AH         LINE#         191
  C:0A3AH         LINE#         192
  C:0A3AH         LINE#         193
  C:0A3CH         LINE#         194
  C:0A3EH         LINE#         196
  C:0A40H         LINE#         197
  C:0A42H         LINE#         198
  C:0A43H         LINE#         199
  C:0A44H         LINE#         200
  C:0A46H         LINE#         202
  C:0A48H         LINE#         203
  C:0A4AH         LINE#         204
  -------         ENDPROC       SETRXMODE
  -------         ENDMOD        NRF2401

  -------         MODULE        ?C?CLDPTR
  C:0A21H         PUBLIC        ?C?CLDPTR
  -------         ENDMOD        ?C?CLDPTR

******************************************************************************
* RESTRICTED VERSION WITH 0800H BYTE CODE SIZE LIMIT; USED: 01DBH BYTE (23%) *
******************************************************************************

Program Size: data=37.1 xdata=0 code=644
LINK/LOCATE RUN COMPLETE.  0 WARNING(S),  0 ERROR(S)
